:038000000283DB1D
:0C83DB00787FE4F6D8FD7581070283B7B7
:10800300000000002E2A3A0088F80000000000005B
:10801300000088FF000000C020C0008088FF00002F
:1080230000010201000088FF0000000000000000C2
:1080330088FF000808002E2A3A00080F08000000F5
:108043000000040000000000020000000000010026
:10805300000000000080000000000040000000005D
:1080630000200000000000100000000000080000D5
:1080730000000004000000000002000000000001F6
:10808300000000000000800000000000400000002D
:1080930000002000000000001000000000000800A5
:1080A30000000000040000000000020000000000C7
:1080B30001000000000000800000000000400000FC
:1080C3000000002000000000001000000000000875
:1080D3000000000000040000000000020000000097
:1080E30000010000000000008000000000004000CC
:1080F300000000002000000000001000000000004D
:10810300080000000000040000000000020000005E
:10811300000001000000000000800000000000409B
:10812300000000000020000000000010000000001C
:02813300000842
:1083B700C29475903E12835B12837D1281D2128222
:0683C700D712830880F8C4
:10828500E4FBFAC293EF70047D0D80027D0FE4FCE0
:10829500C292ED30E304D2918002C291D292ED25D3
:1082A500E0FD0CECB404E9D291C292E4FCEB25E0CC
:1082B500FBEA33FAD292C292EB3091054401FB807E
:1082C5000354FEFB0CECB40CE4D293AF03EA540F59
:0182D500FEAA
:0182D6002285
:1082D700E490E049F0E4FF128285AB07AA067C0030
:1082E7007D6712814790E049E02400F582E434E09D
:1082F700F583EFF090E049E004F0E0C3944940D5FE
:018307002253
:10830800E490E049F090E049E0FEFD3395E0FC742C
:10831800002DF58274E03CF583E0FFEE240AFD129F
:10832800822F90E049E004F0E0C3648094C940D50E
:018338002222
:05822F0090E04AEDF0B3
:10823400A37405F0EF3395E0FE7C007D06128135D2
:10824400A3EEF0A3EFF090E04BE0FDC364809480D4
:10825400402E90E04AE0FF1283CD90E04CE0FEA374
:10826400E0243FF582748012833990E04DE004F0FD
:10827400700690E04CE004F090E04BE014F080C60F
:0182840022D7
:1081D200E490E049F0A3F090E049E0FFA3E0FD1253
:1081E20083CDE490E04BF090E04AE075F00AA49071
:1081F200E04CF090E04CE0FF3395E0FE74032FF585
:1082020082748012833990E04BE004F0A3E004F022
:1082120090E04BE0C36480948A40D8E490E049F057
:0C822200A3E004F0E0D36480948540AB3E
:01822E00222D
:068339003EF583E493FF12
:10833F00D295E4FEEF30E704D2968002C296D29730
:0B834F00C297EF25E0FF0EEEB408E936
:01835A002200
:10839B00C295E4FEEF30E704D2968002C296D297E4
:0B83AB00C297EF25E0FF0EEEB408E9DA
:0183B60022A4
:10835B00C294D2947F2112839B7FBC12839B7F0795
:10836B0012839B7F1312839B7F2012839B7F0C02B4
:02837B00839BE2
:10837D00E4FDFC7F8012839B7F4012839BE4FF1200
:0D838D00833F0DBD00010CBC01F3BDF8F0F5
:01839A0022C0
:0E83CD00EF2480FF12839BED2440FF02839B70
:10813500EF8DF0A4A8F0CF8CF0A428CE8DF0A42E5E
:02814500FE2218
:10814700C2D5EC30E709B2D5E4C39DFDE49CFCEE53
:1081570030E715B2D5E4C39FFFE49EFE12817DC3CD
:10816700E49DFDE49CFC800312817D30D507C3E4C8
:068177009FFFE49EFE22C2
:10817D00BC000BBE0029EF8DF084FFADF022E4CCE6
:10818D00F875F008EF2FFFEE33FEEC33FCEE9DECAF
:10819D00984005FCEE9DFE0FD5F0E9E4CEFD22EDF5
:1081AD00F8F5F0EE8420D21CFEADF075F008EF2F3F
:1081BD00FFED33FD4007985006D5F0F222C398FD30
:0581CD000FD5F0EA22CD
:00000001FF
